:10000000B2014429A2008316051283120930A3000D
:1000100003101120A20CA30B0928031411200314B0
:100020003F2903181628000005163028051230282D
:100030008316861783126400861F1B280030A100D8
:100040001830F9200830A30030200310861F031455
:10005000A20C00002B28A30B242830202208080023
:100060000030A1006230F9280408A70086120612A9
:1000700006128316861206120612F03086058312C7
:100080002708B21861283A30A1009830F92033309F
:10009000A60076201330A1008830F9207620643045
:1000A000F82076206430F8202230A6007620283010
:1000B00060200C30602006306020B21427086128D0
:1000C0003214A600321C6F280612033C031C74284D
:1000D00074201530A1007C30F9200314080032147C
:1000E000FE3C03193F290616A60E321C3210861656
:1000F000F030860526080F3986048612A60E3218BF
:1001000076283230F82003140800B40084178004E5
:100110008413A201201CA200942003193F299420DB
:1001200003193F2994203F293408A2060130A0007A
:10013000A101000834052206031D0800A00A0319C6
:10014000A10F99280800B31329080319B317043025
:10015000A800250EB0202508B020240EB0202408C9
:100160000F39F63E0318073E0A3ED328B313290879
:100170000319B3170530A8002730A3001030CC2096
:100180000330A300E830CC20A3016430CC20A301CD
:100190000A30CC202408D328A2002508A100240876
:1001A000A0001E212008A000A8030319B3132908EA
:1001B0000319DD282802031808002008031DB313C3
:1001C000B31B0800303E3A2983178001840AFF3EA2
:1001D000031DE5283F29A301A200FF30A207031C4D
:1001E000A307031C3F290330A100E330F920ED28C9
:1001F000A101F43EA000A109FE30031C0229A007C2
:100200000318FF28A0076400A10FFF280000201892
:10021000092920180B290800A2000530A80023088E
:100220002102031D15292208200204300318013081
:10023000031902302805031DFF303F29A501A40141
:100240001030A600210DA40DA50D2208A40223083C
:10025000031C230FA502031834292208A40723082E
:100260000318230FA5070310A00DA10DA60B22292B
:1002700020083F29840031088A0030088200831357
:1002800003138312640008008316900183128B010C
:1002900083168C018D010F309C009D018312970104
:1002A0008316C4308500C0308600831283169F01F8
:1002B00083129F0183169B012030840060308312DB
:1002C0008A01E520A030840050308A01E5201030FA
:1002D000840060308A01E4209030840060308A011C
:1002E000E42032308A01EB20851183168511FE301F
:1002F00083128A01352080308A0135204F308A01EF
:10030000352053308A01352043308A013520203092
:100310008A01352020308A01352020308A0135209D
:1003200020308A01352020308A01352020308A0192
:10033000352020308A01352020308A0135202030B8
:100340008A01352020308A01352020308A0135206D
:10035000FE308A013520C0308A01352046308A01BE
:10036000352049308A0135204E308A01352044300D
:100370008A01352045308A01352052308A013520E6
:1003800020308A01352020308A01352020308A0132
:10039000352020308A01352020308A013520203058
:1003A0008A01352020308A01352020308A0135200D
:1003B0000330A300E8308A01EC20C001C10185119F
:1003C00083168511FE3083128A01352080308A0120
:1003D000352050308A01352055308A01352054307F
:1003E0008A01352020308A01352050308A0135209D
:1003F00049308A01352043308A01352020308A0176
:100400003520FE308A013520C0308A013520483041
:100410008A01352049308A01352054308A0135203F
:1004200020308A01352042308A01352055308A013A
:10043000352054308A01352020308A01352064006F
:100440008A11051D6B2A64008A11051D292A8A015B
:10045000232AFE308A01352080308A01352053302E
:100460008A01352054308A01352041308A013520F7
:1004700052308A01352054308A01352049308A01B2
:1004800035204E308A01352047308A013520FE3034
:100490008A013520C0308A01352020308A0135207C
:1004A00020308A01352020308A01352020308A0111
:1004B000352020308A01352020308A013520203037
:1004C0008A01352020308A01352085158316851153
:1004D00083128A116D2A8A01DD290130A0000630BD
:1004E000840040308A0185202008B8002108B90026
:1004F0008A011820C000C101FE308A0135208030F9
:100500008A01352046308A0135203D308A01352068
:1005100020308A013520A9013808A4003908A50037
:100520003430B000B1018A01B62020308A01352074
:1005300020308A013520FE308A013520C0308A0102
:1005400035204F308A01352053308A013520433021
:100550008A0135203D308A0135200230A90040084B
:10056000A4004108A5003430B000B1018A01A320E5
:1005700020308A01352020308A0135203808A0003B
:100580003908A1000730A300D0308A010C218A115C
:10059000031DCC2A8A11CE2A8A016D2A8A111C2BAE
:1005A00064008A11051D1A2B64008A11051D1A2B7F
:1005B000FE308A01352080308A01352041308A01A1
:1005C000352042308A0135204F308A0135205230A3
:1005D0008A01352054308A01352049308A0135207E
:1005E0004E308A01352047308A013520FE308A019D
:1005F0003520C0308A01352020308A013520203056
:100600008A01352020308A01352020308A013520AA
:1006100020308A01352020308A01352020308A019F
:10062000352020308A0135208511831685118312EB
:100630008A01D42A8A016D2AFE308A013520803051
:100640008A01352047308A0135204F308A01352014
:1006500054308A01352020308A01352020308A012B
:1006600035204F308A01352053308A013520433000
:100670008A013520FE308A013520C0308A013520BC
:100680004F308A01352053308A01352043308A01AA
:1006900035203D308A01352024308A013520023052
:1006A000A9004008A4004108A5003430B000B10101
:1006B0008A01A32085118316851164008A11831293
:1006C000051DAB2BFE308A01352080308A01352094
:1006D00052308A01352045308A01352053308A0155
:1006E000352054308A01352041308A01352052307E
:1006F0008A01352054308A01352020308A01352086
:1007000020308A013520FE308A013520C0308A0130
:10071000352057308A01352041308A013520493053
:100720008A01352054308A0135202E308A01352047
:100730002E308A0135202E308A01352020308A0162
:10074000352020308A0135200530A300DC308A01B5
:10075000EC208A01DD2952308A01022055308A01BD
:10076000022049308A01022020308A0102204330D1
:100770008A01022041308A01022042308A0102208F
:1007800052308A01022041308A0102204C308A0115
:0C07900002208A011C2B63008A01CB2B85
:02400E000A3F67
:00000001FF
